:100000000C941E060C941C280C9449280C9446064B
:100010000C9446060C9446060C9446060C94460630
:100020000C9446060C9446060C942C130C9446062D
:100030000C9446060C9446060C9446060C94460610
:100040000C9476280C9446060C94642C0C94A72CE3
:100050000C9446060C9446060C9446060C944606F0
:100060000C9446060C944606B5181719F618F9189C
:10007000FC18FF1802190519081917191119491A3E
:100080004B1A4B1A491A4B1A4B1A4B1A4B1A4B1A4A
:100090004B1A4B1A4B1A4B1A4B1A4B1A4B1A4B1A38
:1000A000CF194B1A4B1A4B1A4B1A4B1A40194B1AB1
:1000B0004B1A4B1A4B1A4B1A4B1A4B1A4B1A4B1A18
:1000C0004B1A4B1A4B1A4B1A4B1A4B1ADB19DB19EA
:1000D000DB19DB19DB19DB19DB19DB19DB194B1A0F
:1000E0004B1A4B1A4B1A4B1A4B1A4019DA19DA19D8
:1000F000DA19DA194B1AE819EE19F419FA19001A73
:10010000061A0C1A121A1C1A261A301A3A1A8119CF
:1001100043194B1A4B1A4B1A4B1ACF194B1A4B1A3D
:100120004B1A4B1A4B1A4B1A4B1A4B1AD919D9198D
:10013000D919D9194B1AE819EE19F419FA19001A34
:10014000061A0C1A121A1C1A261A301A3A1A81198F
:1001500043194B1A4B1A4B1A4B1ACF197E1A7E1A97
:100160007E1A7E1A7E1A7E1A7E1A7E1A7E1A7E1ACF
:100170007E1A7E1A7E1A951B951B951B951B951B47
:10018000951BC31ACD1AD71AE11A3F1B491B581BDE
:10019000691BF11C061D121D1B1D2A1D4F1D581D1C
:1001A000A11D6A1DB320B920BF20C620D420F6208F
:1001B0001421456E746572206D656E752E2E2E00AD
:1001C000546F67676C6564206D6963726F50504D42
:1001D00000546F67676C656420696E76657274653C
:1001E000642050504D2100546F67676C6564205443
:1001F00058206D7574696E672100546F67676C6570
:10020000642074656C656D65747279210050726F3D
:10021000746F636F6C206572726F72207769746897
:100220002052580054696D656F7574207768656E4B
:1002300020636F6E6E656374696E6720746F205201
:100240005800507265737320616E79206B65792058
:10025000746F2063616E63656C00436F6E6E6563DF
:1002600074696E6720746F2052582C20706F776508
:100270007220757020746865205258202877697440
:10028000682062696E6420706C7567206966206EF4
:100290006F74207573696E6720616C776179732064
:1002A00062696E642900546F67676C656420276912
:1002B0006D6D656469617465206F75747075742700
:1002C00000546F67676C65642027736C61766520E6
:1002D0006D6F64652700546F67676C6564202761E4
:1002E0006C776179732062696E642700546F676769
:1002F0006C65642050504D206368616E6E656C20A3
:100300006C696D69740053657420525353492069B8
:100310006E6A656374696F6E206368616E6E656C8A
:100320002028303D3D64697361626C652900536526
:10033000742050504D206D696E696D756D20737914
:100340006E630053657420626561636F6E20696E31
:1003500074657276616C0053657420626561636FC9
:100360006E2064656C617900536574206265616319
:100370006F6E206672657175656E637920696E2097
:10038000487A3A20303D64697361626C652C205074
:10039000783D504D52206368616E6E656C20782CFC
:1003A0002046783D465253206368616E6E656C202E
:1003B00078005365742050574D2073746F7020641B
:1003C000656C61792028302064697361626C6564B2
:1003D0002C20312D323535203D3D20302E317320FB
:1003E0002D2035306D696E29005365742050504DB5
:1003F0002073746F702064656C61792028302064EC
:10040000697361626C65642C20312D323535203D75
:100410003D20302E3173202D2035306D696E29003E
:10042000536574206661696C736166652064656CF0
:1004300061792028302064697361626C65642C20C6
:10044000312D323535203D3D20302E3173202D2089
:1004500035306D696E29002A2A2A2A2A2A2A2A2A50
:100460002A2A2A2A2A2A2A2A2A2A2A2A2A2A2A2AEC
:100470002A2A2A2A0052582041636B6564202D20C5
:1004800072657665727420737563636573736675E0
:100490006C21002A2A2A2A2A2A2A2A2A2A2A2A2AAD
:1004A0002A2A2A2A2A2A2A2A2A2A2A2A2A2A2A2AAC
:1004B000002A2A2A2A2A2A2A2A2A2A2A2A2A2A2AC6
:1004C0002A2A2A2A2A2A2A2A2A2A2A2A2A2A00528E
:1004D000582041636B6564202D20757064617465DC
:1004E000207375636365737366756C21002A2A2A0D
:1004F0002A2A2A2A2A2A2A2A2A2A2A2A2A2A2A2A5C
:100500002A2A2A2A2A2A2A2A2A2A0056616C696457
:100510002063686F69636573206172653A205B319F
:100520005D2D5B31365D20286368616E6E656C20E1
:10053000312D31362900536574206F7574707574D0
:1005400020666F7220706F727420005B585D2061AE
:10055000626F7274206368616E67657320616E6498
:10056000206578697420525820636F6E6669670051
:100570005B535D20736176652073657474696E6783
:100580007320746F205258005B525D20726576654F
:1005900072742052582073657474696E6773207486
:1005A0006F2064656661756C747300557365206EA9
:1005B000756D62657273205B312D445D20746F2010
:1005C0006564697420706F727473205B452D515D92
:1005D00020666F722073657474696E677300202DD6
:1005E00020726563656976657220636F6E66696700
:1005F000757261746F722C20727820737720000AF4
:100600000A6F70656E4C52536E67200053657420FC
:1006100073657269616C2062617564726174653AB8
:10062000200056616C69642063686F696365733A82
:100630002031202D20342B34202F2032202D203823
:10064000202F2033202D20382B34202F2034202D14
:10065000203132202F2035202D2031322B34202FF5
:100660002036202D20313600536574204368616E9A
:100670006E656C20636F6E6669673A20005365741F
:100680002044617461726174652028302D32293AEA
:10069000200053657420486F70206368616E6E653A
:1006A0006C7320286D61782032342C207365706162
:1006B000726174656420627920636F6D6D61732966
:1006C0002076616C69642076616C75657320312DCC
:1006D0003235353A2000536574206368616E6E656B
:1006E0006C2073706163696E6720287831306B48C5
:1006F0007A293A200053657420524620706F77653E
:10070000722028302D37293A200053657420524634
:10071000206D6167696320286865782920652E67E8
:100720002E20307844454144463030443A2000532E
:1007300065742062617365206672657175656E63AC
:10074000792028696E20487A293A20005B5A5D207A
:10075000656E746572207265636569766572206383
:100760006F6E66696775726174696F6E2075746902
:100770006C79005B465D20646973706C61792061FF
:10078000637475616C206672657175656E63696509
:10079000732075736564005B525D2063616C6375E3
:1007A0006C6174652072616E646F6D206B65792079
:1007B000616E6420686F70206C697374005B495DC2
:1007C000207265696E697469616C697A6520736508
:1007D0007474696E677320746F20736B65746368DB
:1007E0002064656661756C7473005B585D2072658A
:1007F00076657274206368616E67657320616E64EC
:100800002065786974206D656E75005B535D20739B
:100810006176652073657474696E677320746F20E8
:10082000454550524F4D20616E64206578697420B3
:100830006D656E7500557365206E756D62657273BA
:10084000205B302D395D20746F20656469742070E1
:100850006172616D657465727300202D2053797328
:1008600074656D20636F6E66696775726174696F18
:100870006E000A0A6F70656E4C52536E672000510D
:1008800029204F7574707574206265666F726520DB
:100890006C696E6B20283D465329203A2000502970
:1008A00020536C617665206D6F64652028657870D3
:1008B0006572696D656E74616C293A20004F29205C
:1008C00054696D65642042494E44206174207374FC
:1008D000617274757020203A20004E292050504DCE
:1008E000206F7574707574206C696D69746564200F
:1008F000202020203A200044495341424C454400E6
:100900004D292050504D205253534920746F20637D
:1009100068616E6E656C202020203A20004C2920F2
:1009200050504D206D696E696D756D2073796E63E1
:10093000202875732920203A200044495341424C15
:100940004544004B29204661696C736166652062ED
:100950006561636F6E20696E74762E2028312D32AA
:10096000353573293A20004A29204661696C736144
:10097000666520626561636F6E2064656C617920D5
:1009800028302D323535203D3E20313073202D204A
:100990003135306D696E293A200049292046616958
:1009A0006C7361666520626561636F6E206672714B
:1009B0002E203A200048292050574D2073746F7024
:1009C0002064656C6179202020202020203A2000BE
:1009D00047292050504D2073746F702064656C61FE
:1009E00079202020202020203A200046292046611E
:1009F000696C736166652064656C617920202020D4
:100A00002020203A200050574D206368616E6E65AB
:100A10006C200066756E6374696F6E3A2000292041
:100A2000706F72742000506F776572546F776572C3
:100A300000445446205548462033322D62697420C4
:100A400031306368004F70656E4C52536E67525878
:100A5000206D696E6920342F36636800466C7974A6
:100A6000726F6E2F4F72616E6765525820554846FF
:100A70002038636800525820747970653A20004429
:100A8000697361626C656400487A00203D3D200016
:100A900043616C63756C61746564207061636B6540
:100AA0007420696E74657276616C3A200042292068
:100AB0004D6963726F202868616C66292050504D23
:100AC000202020203A00412920496E766572746505
:100AD000642050504D20696E20202020203A0030A4
:100AE00029204D7574652062757A7A657220286DAB
:100AF0006F73746C79293A003929205365726961E2
:100B00006C2062617564726174653A00736D617224
:100B100074506F7274004672536B79005472616E38
:100B200073706172656E740044697361626C6564B0
:100B30000038292054656C656D657472793A2020FF
:100B40002020202020003729204368616E6E656CCC
:100B500020636F6E6669673A202000362920446161
:100B60007461726174652028302D32293A2020206A
:100B700000352920486F70206368616E6E656C7364
:100B80003A2020202020003429204368616E6E65C1
:100B90006C2073706163696E673A202000332920EE
:100BA000524620706F7765722028302D37293A2001
:100BB0002020003229205246206D616769633A2067
:100BC0002020202020202020003129204261736530
:100BD000206672657175656E63793A202020000089
:100BE00000000700020100000304060000000000EE
:100BF00000000001020408102040800102040810D7
:100C00002001020408102004040404040404040263
:100C10000202020202030303030303000000002395
:100C2000002600290000000000250028002B0000FD
:100C3000000000240027002A0000952D11241FBE6B
:100C4000CFEFD8E0DEBFCDBF13E0A0E0B1E0E8E336
:100C5000F1E602C005900D92A83CB107D9F716E065
:100C6000A8ECB3E001C01D92AE38B107E1F71CE07B
:100C7000CCE3DCE004C02297FE010E949E2ECA3322
:100C8000D107C9F70E94D12D0C949A300C94000022
:100C900080917305813019F482E08093730580910F
:100CA0007305833019F484E0809373050895A89543
:100CB0000895DC01ED91FC910190F081E02D099502
:100CC00008952091740530917505382748E0C901D1
:100CD000880F991F37FF06C09C0151E2252750E17C
:100CE000352701C09C01415091F730937505209341
:100CF0007405089588E38093760580E092ECA1E086
:100D0000B0E08093770590937805A0937905B09330
:100D10007A0587E08093830580EC92E9ADEEB9E136
:100D200080937B0590937C05A0937D05B0937E0511
:100D300085E0809384058DEE9EEFADEABEED809355
:100D40007F0590938005A0938105B0938205E5E827
:100D5000F5E080E090E0863028F4DC01AE54BC4F32
:100D60002C9101C020E0219301968831910599F7DB
:100D700082E080939D058AE080939E05089580EC33
:100D800091EDA8E9BBE18093BB059093BC05A093CE
:100D9000BD05B093BE0580E090E0A0E0B0E5809393
:100DA000BF059093C005A093C105B093C205E3ECC5
:100DB000F5E080E081938F5F8031E1F70895A0E056
:100DC000B0E0E5EEF6E00C94672ED82F0E94CC2818
:100DD0006115710581059105C9F30E940A2F1092D2
:100DE0007F05109280051092810510928205C4E063
:100DF000812C912C54018A94C0907F05D09080055D
:100E0000E0908105F0908205FE2CED2CDC2CCC24AA
:100E10000E94052FA50194010E94462E6C0D7D1D98
:100E20008E1D9F1D60937F057093800580938105C3
:100E300090938205C15001F7DD2309F450C005E805
:100E400015E0E801A12CB12C62E3C62ED12CE12CD7
:100E5000F12C8881882309F442C0B39419F40E94CC
:100E60007A063DC00E94052FA70196010E94462EDA
:100E7000E1E0E60FA5E8B5E08A2F801B8A1520F493
:100E80008D918E13F9CFE9CF2091840530E0A0E158
:100E9000B7E20E94DE2D9B01AC01AE2FB0E00E94B4
:100EA000ED2D40907B0550907C0560907D05709005
:100EB0007E05640D751D861D971D4090BB055090E5
:100EC000BC056090BD057090BE05461657066806C5
:100ED000790618F2E993A39488E1A812BACFCDB7A6
:100EE000DEB7E0E10C94832E8436910520F4BC013A
:100EF00080E090E017C09C018E3B910528F42A55B4
:100F00003109AAE0B0E00CC0823D910528F4245BD1
:100F10003109A4E6B0E004C02D5C3109A8E5B2E0D7
:100F20000E94DE2DA4E6B0E09B01AC010E94ED2DF5
:100F3000089590E08C599F4F0E947407089561E0D6
:100F400083E10E94792960E083E10E94B22982E076
:100F50008093B00085E08093B10061E083E00E945F
:100F6000792960E083E00E94B2290895A4E0B0E00E
:100F7000ECEBF7E00C94752E009749F19C0140E0F2
:100F800050E068E478EE81E090E00E94462E61E057
:100F900083E129833A834B835C830E94B2292981B0
:100FA000822F3A81932F4B81A42F5C81B52F8F3FE5
:100FB0009105A105B10529F020F08FEF90E0A0E0A8
:100FC000B0E08093B3008091B000806107C060E022
:100FD00083E10E94B2298091B0008F7E8093B0009F
:100FE0002496E2E00C94912E60E08CE00E94792936
:100FF00061E08BE00E94792961E08DE00E9479290F
:1010000060E082E00E94792961E084E00E94792911
:10101000089542E050E068E476E080E00E94FC271A
:101020000895E3E0F0E089E080935700E491E670F2
:1010300081E0E63009F080E00895CF93DF93C82F78
:101040000E941108882381F0DFB781E08093720548
:10105000F8940E94570688E180936000C093600076
:10106000C1110E945706DFBFDF91CF9108958F9283
:101070009F92AF92BF92CF92DF92EF92FF92CF9367
:10108000FC01C0A5EC2FE770F0E0E658FC4FA08112
:10109000B0E0C7FF03C024E130E002C02FE030E041
:1010A000FC0197A183E1989FF0011124E25CFE4FBF
:1010B00080809180A280B380A20FB31F20E43FE123
:1010C0004DE750E00E94F82DA50194010E94242EC6
:1010D0008C2F887149F469017A01E0EDCE0EE7E0CA
:1010E000DE1EE11CF11C1BC0C7FF05C060E47AE8EE
:1010F0008CE29EE004C060E07EEE8AEB9BE069013A
:101100007A01F8EBCF0EFBE0DF1EE11CF11CA5011C
:1011100094010E94242EC20ED31EE41EF51EC701A8
:10112000B60169517C4F8F4F9F4F28EE33E040E06E
:1011300050E00E94242EA8EEB3E00E94ED2DCF9146
:10114000FF90EF90DF90CF90BF90AF909F908F90E7
:1011500008958F3F910551F048F0811522E09207E4
:1011600038F08115934030F482E0089580E00895CE
:1011700081E0089583E00895A0E0B0E0E2ECF8E0BB
:101180000C94702EEB018A01B82FB695A0E028814F
:101190003981F80120832A813B8121832C813D8183
:1011A00022832E813F812383688179814A815B81FB
:1011B0002C813D81EE81FF819F2F9295990F990F90
:1011C000907C272F2370922B252F2370220F220F24
:1011D000922B232F23702295207F922BF80194834A
:1011E0000B5F1F4F2896AF5FBA1788F680FF24C0A9
:1011F000888199810E94A908D82E8A819B810E94AA
:10120000A908E82E8C819D810E94A908F82E8E8164
:101210009F810E94A908F0E4DF9EA001112490E1C3
:10122000E99E90011124242B282BE4E0FE9EB001BE
:101230001124262BF8012083CDB7DEB7E7E00C940C
:101240008C2E803223E0920708F1883E23E092073B
:1012500040F48F519340E4E096958795EA95E1F745
:101260000895803D27E0920718F48C5D934008951F
:10127000883928E0920768F4885C974074E0969576
:1012800087957A95E1F78D509C4F089580E090E026
:1012900008958FEF93E008958C30910540F4A4E019
:1012A000880F991FAA95E1F7885D9C4F0895843FA8
:1012B00023E0920718F484529C4F0895811524E08E
:1012C000920740F48657934FF4E0880F991FFA95E0
:1012D000E1F7089580E998E008959C0136952795F7
:1012E00025753575821B930B9C012373337396957B
:1012F00087959695879583739373820F931F9C01AF
:1013000054E0369527955A95E1F7280F391F2F702D
:101310003F7041E051E0249FC001259F900D349F14
:10132000900D1124892F08952D98882319F000001D
:101330002B9A02C000002B9800002D9A00000895FF
:101340002D9A000083B12D98000082958170089538
:10135000CF93DF93D82F5C9A2D985C98C8E08D2F9F
:1013600080780E949409DD0FC150C9F72D98DF9154
:10137000CF9108958F770E94A8090895CF93DF93A6
:10138000D82FC8E08D2F80780E949409DD0FC150BE
:10139000C9F72D98DF91CF910895CF93DF932D98C2
:1013A000C8E080E0D82FDD0F0E94A0098D0FC1504A
:1013B000C9F7DF91CF9108950E94BA090E94CD0923
:1013C0005C9A0895A1E0B0E0E8EEF9E00C94752E87
:1013D000806869830E94A8096981862F0E94BE09DE
:1013E0005C9A2196E2E00C94912ECF93C0917F05F8
:1013F000C827E82FF0E0EA58FA4F678589E70E948E
:10140000E2096C2F8DE30E94E2096C2F82E40E94B6
:10141000E209CF91089586E20E94DC090895CF93F6
:10142000DF93EC016C818CE10E94E2096D818DE11A
:101430000E94E2096E818EE10E94E2096F8180E2E2
:101440000E94E209688581E20E94E209698582E2E0
:101450000E94E2096A8583E20E94E2096B8584E2C8
:101460000E94E2096C8585E20E94E2096D858AE2AC
:101470000E94E2096E858EE60E94E2096F858FE682
:101480000E94E209688980E70E94E209698981E790
:101490000E94E2096A8982E70E94E209DF91CF9106
:1014A0000895CF92DF92EF92FF92CF93DF936B017B
:1014B0007C01C11488E3D8068CE9E8068CE1F806C3
:1014C00028F5C701B60120E836E948E950E00E9456
:1014D000242EE901689760E879E687E69FEF0E948D
:1014E000002E6C0D7D1D8E1D9F1DF2E0660F771F77
:1014F000881F991FFA95D1F721E732E040E050E0CC
:101500000E94242EF22EE32E80E421C0C701B601F2
:1015100020E03DE241E351E00E94242EE90168977A
:1015200060E073ED8EEC9EEF0E94002E6C0D7D1D31
:101530008E1D9F1D660F771F881F991F21E732E0C0
:1015400040E050E00E94242EF22EE32E80E66C2F25
:101550006F71680F85E70E94E2096E2D86E70E9491
:10156000E2096F2D87E70E94E209DF91CF91FF909A
:10157000EF90DF90CF900895682F8DE60E94E209EA
:1015800008958F929F92AF92BF92CF92DF92EF9287
:10159000FF92CF93DF93D82F83E00E94DC098093E2
:1015A000710584E00E94DC098093700560E086E0AC
:1015B0000E94E20961E087E00E94E2096FE789E0AA
:1015C0000E94E20965E08AE00E94E20962E18BE0A4
:1015D0000E94E20965E18CE00E94E2096DEF8DE076
:1015E0000E94E20960E08EE00E94E209DD2319F02A
:1015F0008BE291E008C020919D0533E1239FC0015B
:101600001124825C9E4F0E940F0A6CE880E30E94C6
:10161000E2096FE082E30E94E20962E483E30E9450
:10162000E20980919E0587FF02C064E101C06AE083
:1016300084E30E94E2096AE285E30E94E2096DE226
:1016400086E30E94E20964ED87E30E94E20960E01C
:1016500088E30E94E20960E089E30E94E209D11177
:1016600009C0C0907F05D0908005E0908105F09082
:10167000820507C0C5E9CC2EC1ECDC2EED2CCEEDE9
:10168000FC2ECAE38F2C9924AA24BB24682D8C2F0E
:101690000E94E209682D85E08C0F0E94E209FE2C71
:1016A000ED2CDC2CCC24CF5FCE3361F76FEF83E4DD
:1016B0000E94E2096FEF84E40E94E2096FEF85E483
:1016C0000E94E2096FEF86E40E94E209DD2311F037
:1016D00066E002C0609183058DE60E94E20960E049
:1016E00089E70E94E209609184058AE70E94E20985
:1016F00060E083E70E94E20960E084E70E94E2097B
:10170000D11109C060917B0570917C0580917D05A8
:1017100090917E0504C060EC72E98DEE99E10E9423
:10172000510ADF91CF91FF90EF90DF90CF90BF9063
:10173000AF909F908F90089561E087E00E94E2094A
:1017400064E28EE70E94E20963E088E00E94E20919
:1017500060E088E00E94E20965E087E00E94E2091B
:1017600062E085E00E94E20983E00E94DC09809348
:10177000710584E00E94DC0980937005089583E080
:101780000E94DC098093710584E00E94DC0980934B
:10179000700561E087E00E94E2096AE070E080E0A5
:1017A00090E00E94EF280E949C0B00000895CF92C9
:1017B000DF92FF920F931F93CF93DF931F92CDB7CA
:1017C000DEB7082F162F8EE399830E94E209F02ED0
:1017D000C02E9981D92E8C2D8F19811738F4F601DE
:1017E00061916F018FE70E94E209F5CF64E085E027
:1017F0000E94E20983E00E94DC098093710584E085
:101800000E94DC09809370050E94CC2860936C05CF
:1018100070936D0580936E0590936F0569E087E086
:101820000E94E20981E0809373050F90DF91CF91D0
:101830001F910F91FF90DF90CF9008950F931F930A
:101840000E94D70B80917305813099F40E94CC28B7
:1018500000916C0510916D0520916E0530916F051A
:10186000601B710B820B930B603A764881409105A7
:1018700048F380917305813031F46EE971E082EEB6
:1018800095E00E94B82A1F910F9108950F931F931E
:1018900080917305823021F41092730581E020C09D
:1018A000809173058130D9F40E94CC2800916C0599
:1018B00010916D0520916E0530916F05601B710BC5
:1018C000820B930B613A76488140910540F061E0CC
:1018D00087E00E94E2091092730582E001C080E077
:1018E0001F910F910895CF93DF93EC014AE050E0F0
:1018F0006D2F70E082EE95E00E94862B6EE282EE04
:1019000095E00E948A2ABE0184E0769567958A95C3
:10191000E1F76F7077274AE050E082EE95E00E9491
:10192000862B6EE282EE95E00E948A2ABE016F70DD
:1019300077274AE050E082EE95E00E94862BDF9107
:10194000CF910895D82FC0E0CD1780F4439A64E674
:1019500070E080E090E00E94EF28439864E670E039
:1019600080E090E00E94EF28CF5FEECF6CE271E064
:1019700080E090E00E94EF28E6CF0F931F93CF9373
:10198000DF93EC01062F15E0115051F0CE010E94BB
:101990008130081741F0602FCE010E948930F4CFCA
:1019A00082E00E94A20CDF91CF911F910F910895C8
:1019B000A0E0B0E0EEEDFCE00C94672E482E562E31
:1019C000C0E0D0E0612C712CE12CF12C00E010E0A3
:1019D00041100CC06090D40586E4689E300111244B
:1019E00059E1E52EF12C0AEB15E01EC091E04912F9
:1019F0000FC06090D405E6E46E9E30011124FBE137
:101A00006F0E711C49E2E42EF12C06E715E00CC0C4
:101A100082E0481209C028E1622E77247394EE24F4
:101A2000E394F12C03ED15E043018C0E9D1E109202
:101A30007505109274053401A62CA818B12CC301A9
:101A400001966C01AE14BF04A8F4A00EB11E511093
:101A500006C0C3010E948130F501808305C0F501F5
:101A60006081C3010E94BD0CF50180810E94610666
:101A70003601E2CFC301511018C0C3010E9481306A
:101A8000B82EC6010E9481302B2D30E0322F222744
:101A9000282B80917405909175058217930779F42E
:101AA000C0E0D0E05524539493CF36016091750582
:101AB0000E94BD0C60917405C6010E94BD0CC05E01
:101AC000DE4FC13E92E0D90708F482CF852DCDB715
:101AD000DEB7E0E10C94832E61E082E00E94D80C36
:101AE000089560E082E00E94D80C8091D305853093
:101AF00020F01092D3050E946C0D8091D305809345
:101B0000D405089561E080E00E94D80C61E081E096
:101B10000E94D80C089560E080E00E94D80C8823D1
:101B200051F060E081E00E94D80C882321F0809180
:101B30007605883349F00E94BF060E947A0681E04C
:101B40000E94DF060E94820D0895882319F06AEA38
:101B500071E002C06EEA71E082EE95E00E94B82A60
:101B60000895FF920F931F93CF93DF9369EC7BE06F
:101B700082EE95E00E94642A40917B0550917C059D
:101B800060917D0570917E052AE030E082EE95E05F
:101B90000E948D2B63EB7BE082EE95E00E94642A2D
:101BA00040917F055091800560918105709182057B
:101BB00020E130E082EE95E00E948D2B6DE97BE024
:101BC00082EE95E00E94642A4AE050E0609183052D
:101BD00082EE95E00E94B52B67E87BE082EE95E00F
:101BE0000E94642A4AE050E06091840582EE95E00C
:101BF0000E94B52B61E77BE082EE95E00E94642AAB
:101C0000C5E8D5E0F12C8E0188818823A9F0FF205A
:101C100031F061EB71E082EE95E00E94872A219617
:101C20004AE050E0F801608182EE95E00E947E2B50
:101C3000F394F8E1FF12E7CF82EE95E00E94922A3A
:101C40006BE57BE082EE95E00E94642A4AE050E07A
:101C500060919D0582EE95E00E94B52B66E47BE0E5
:101C600082EE95E00E94642AE0919E05E770F0E024
:101C7000EE0FFF1FEE57FC4F6081718182EE95E001
:101C80000E94B82A61E37BE082EE95E00E94642A1C
:101C900080919E058871883069F028F4811113C005
:101CA00068E27BE00CC0803141F0883161F46CE087
:101CB0007BE005C06CE17BE002C066E17BE082EE88
:101CC00095E00E94A62A68EF7AE082EE95E00E94F5
:101CD000642A40917705509178056091790570915B
:101CE0007A052AE030E082EE95E00E948D2B6FEDC0
:101CF0007AE082EE95E00E94642A8091BF058071AF
:101D00000E94A50D66EC7AE082EE95E00E94642ABE
:101D10008091BF0580740E94A50D6DEA7AE082EE85
:101D200095E00E94642A8091BF0580720E94A50DF3
:101D300060E97AE082EE95E00E94642A86E795E009
:101D40000E943708AB01BC012AE030E082EE95E04A
:101D50000E946F2B6BE87AE082EE95E00E94642A85
:101D600086E795E00E9437089B01AC0160E472E4CD
:101D70008FE090E00E94242EBA01A9012AE030E011
:101D800082EE95E00E946F2B68E87AE082EE95E0A3
:101D90000E94A62ACDB7DEB7E5E00C948E2E8F9276
:101DA0009F92AF92BF92CF92DF92EF92FF928111FA
:101DB00007C06FE77AE082EE95E00E94A62A2FC066
:101DC00090E00E94740724E630E040E050E00E947A
:101DD000242ECA01B9012AE030E040E050E00E9420
:101DE000242E49015A016B017C012AE030E0B50143
:101DF000A40182EE95E00E946F2B6EE282EE95E0E8
:101E00000E948A2A2AE030E0B701A60182EE95E01E
:101E10000E946F2B63E782EE95E00E94CA2AFF9032
:101E2000EF90DF90CF90BF90AF909F908F900895EC
:101E30001F93CF93DF9365E77AE082EE95E00E94EF
:101E4000642A80919F05813041F46CE57AE082EE4E
:101E500095E00E94A62A10E050C0823019F465E493
:101E60007AE0F5CF843019F461E37AE0F0CF853081
:101E700091F766E27AE0EBCFC12FD0E0C930D1050F
:101E80000CF441C068E3610F82EE95E00E948A2A5B
:101E90006EE17AE082EE95E00E94642ABE016F5FF7
:101EA0007F4F4AE050E082EE95E00E944E2B63E1C6
:101EB0007AE082EE95E00E94642AC156DA4FE98109
:101EC000E03218F566E07AE082EE95E00E94642A3E
:101ED0008981803130F06DE673E082EE95E00E94FA
:101EE000872A69816F7070E06F5F7F4F4AE050E032
:101EF00082EE95E00E94572B1F5F809148051817CE
:101F000008F4BACF0FC061E3BECFEF70F0E0EE0F80
:101F1000FF1FEE56FC4F6081718182EE95E00E94BA
:101F2000B82AEACF6BEE79E082EE95E00E94642A4F
:101F30008091B7050E94CF0E60ED79E082EE95E0CA
:101F40000E94642A8091B8050E94CF0E65EB79E06B
:101F500082EE95E00E94642A8091B9050E94CF0E1E
:101F60006AE979E082EE95E00E94642A4091AF052B
:101F70005091B0056091B1057091B20541155105C0
:101F80006105710539F12AE030E082EE95E00E94AA
:101F90008D2B67E679E082EE95E00E94642A8091BD
:101FA000B3050E949907AB01BC012AE030E082EE44
:101FB00095E00E948D2B63E479E082EE95E00E942B
:101FC000642A4AE050E06091B40582EE95E00E94F8
:101FD000B52B06C06AE379E082EE95E00E94A62A5E
:101FE0006DE179E082EE95E00E94642A6091B5058A
:101FF0007091B6054AE050E082EE95E00E949F2B7A
:1020000060E079E082EE95E00E94642A6091AE057E
:10201000603450F470E06F5F7F4F4AE050E082EE32
:1020200095E00E94572B06C067EF78E082EE95E0BE
:102030000E94A62A6AED78E082EE95E00E94642A6A
:102040008091AD0580FF03C063EB71E002C067EBD8
:1020500071E082EE95E00E94B82A6DEB78E082EEA6
:1020600095E00E94642A8091AD0582700E94A50DC2
:102070006EE978E082EE95E00E94642A8091AD05D9
:1020800084700E94A50D6FE778E082EE95E00E94D3
:10209000642A8091AD0588700E94A50DDF91CF91D3
:1020A0001F9108950F931F93CF93DF9320914505C0
:1020B0002F3FA9F56FEF75E082EE95E00E94642A4C
:1020C00084E893E00E94730C6EED75E082EE95E07B
:1020D0000E94642A80914605909147050E94730CE6
:1020E0006BEA75E082EE95E00E94A62A68E875E04A
:1020F00082EE95E00E94A62A60E775E082EE95E008
:102100000E94A62A6BE475E082EE95E00E94A62A62
:1021100082EE95E00E94922A0E94180F68C0121663
:102120000CF065C0332727FD30958091480590E07D
:10213000821793070CF45BC066E375E082EE95E0CE
:102140000E94642A60914505772767FD70954AE0F3
:1021500050E082EE95E00E94572B6BE075E082EE36
:1021600095E00E94642A10E008E280914905181762
:10217000D0F5C12FD0E0CC0FDD1FC65BDA4F288130
:1021800030E080914505992787FD909501972817A4
:10219000390739F56BEB71E082EE95E00E94872AF2
:1021A0004AE050E0602F82EE95E00E947E2B6FEBBC
:1021B00071E082EE95E00E94872AE981EF70F0E0FD
:1021C000EE0FFF1FEE56FC4F6081718182EE95E0AD
:1021D0000E94872A63EC71E082EE95E00E94872AD4
:1021E0000F5F1F5FC2CF82EE95E00E94922ADF91BF
:1021F000CF911F910F910895FF920F931F93CF934B
:10220000DF93C5E8D5E0F12C8E0188818823D1F1D8
:1022100065EC71E082EE95E00E94872A4AE050E08A
:102220006F2D82EE95E00E947E2B62ED71E082EED2
:1022300095E00E94872A2196F801208130E0A0E1F4
:10224000B7E20E94DE2D9B01AC01A0918405B0E0B5
:102250000E94ED2DAB01BC0180917B0590917C0526
:10226000A0917D05B0917E05480F591F6A1F7B1F05
:102270002AE030E082EE95E00E948D2BF394F8E1A5
:10228000FF12C2CFCDB7DEB7E5E00C948E2E1092D0
:10229000DF0485E6E0EEF4E0DF011D928A95E9F7C0
:1022A0000895CF93C82F8F3719F0883009F045C0B3
:1022B000E091DF04EE23D9F1E150E093DF04F0E098
:1022C000E052FB4F10826DE070E082EE95E00E94DC
:1022D0005906C0E08091DF04C81760F4EC2FF0E0ED
:1022E000E052FB4F608170E082EE95E00E9459065B
:1022F000CF5FF0CF60E270E082EE95E00E94590679
:102300006DE070E082EE95E00E945906C0E0809199
:10231000DF04C81778F5EC2FF0E0E052FB4F608146
:1023200070E082EE95E00E945906CF5FF0CF67E043
:1023300082EE95E00E948A2A1DC08B3119F40E941A
:1023400047111AC08D30C1F08A30B1F08091DF049E
:10235000843668F76C2F70E082EE95E00E94590693
:10236000E091DF0481E08E0F8093DF04F0E0E05223
:10237000FB4FC08380E001C081E0CF910895CF93EF
:10238000C82F0E94CC286093C8047093C90480931E
:10239000CA049093CB04C093DD04CC2329F040E021
:1023A00051EE60E070E004C040E855E260E070E0AB
:1023B00082EE95E00E94142DCF9108959091CC0467
:1023C000492F4F7050E0BA016F5F7F4F292F30E0E7
:1023D000E4E035952795EA95E1F76217730759F020
:1023E000FA01E353FB4F808381E0890F8F70907F68
:1023F000892B8093CC0408956EE770E082EE95E01F
:102400000E9459060895A3E1B1E0E9E0F2E10C94DD
:10241000682EE5E8F5E0712C8191882321F0739412
:1024200028E17212F9CF66ED71E082EE95E00E942C
:10243000B82A4AE050E0672D82EE95E00E94B52B65
:1024400080E00E94C10A0E949C0B8E010E5F1F4F0C
:10245000C12CD12C7601C39466246A945C2C0E9412
:10246000C0284B015C012091840530E0A0E1B7E277
:102470000E94DE2D9B01AC01C701B6010E94002E17
:1024800020917B0530917C0540917D0550917E0522
:10249000620F731F841F951F2091BB053091BC05EF
:1024A0004091BD055091BE052617370748075907CB
:1024B00018F4F801608225C08C2D0E94F50961E0B6
:1024C00070E080E090E00E94EF28F80110820E9406
:1024D000C028681979098A099B09643F7140810500
:1024E000910540F40E940B0AF8019081981778F743
:1024F0008083EDCF50FE03C04298439A02C0429AB7
:1025000043982FEFC21AD20AE20AF20A0F5F1F4F56
:102510008FEFC816D104E104F10409F09FCFCE017A
:102520009395FC01D82E7FEF68EC2E2F281B2715E2
:1025300010F051E056C0DE01129651E02FEF41E05D
:102540003D91321710F0322F01C0452F5F5F5F3F82
:1025500011F0232FF5CF4193242F30E0A1E0B0E01C
:10256000AC0FBD1FA20FB31F5C93413079F0DE01A9
:10257000A20FB31F5C93423049F0AFEFBFEFAC0F37
:10258000BD1FA20FB31F6C934E3F78F6A2E0B0E0E0
:10259000AC0FBD1FA20FB31F7C934D3F30F6A3E0DD
:1025A000B0E0AC0FBD1FA20FB31F6C93BECF452F81
:1025B000242F30E0FC01E20FF31F6081AFEFB0E0A9
:1025C000AC0FBD1FA20FB31F2C91621748F44150EE
:1025D000DC01A40FB11D2C9120836C934111E8CF35
:1025E0005F5F571520F3372D369520E0231770F4E1
:1025F000DC01A20FB11D4C91522F530FFC01E50FCE
:10260000F11D50815C9340832E5FF0CFF5E8EF2EF3
:10261000F5E0FF2E8C01802F8D19871598F4F801B5
:10262000C1908F014AE050E06C2D82EE95E00E944F
:102630007E2B6CE282EE95E00E948A2AF701C1921D
:102640007F01E9CF82EE95E00E94922A81E0CD5E83
:10265000DE4FEFE00C94842E1F920F920FB60F9274
:1026600011241F932F933F934F935F936F937F9307
:102670008F939F93AF93BF93CF93DF93EF93FF938A
:10268000C0918600D0918700809187049091880442
:102690002091A904211155C09E01281B390B80915E
:1026A000BF059091C005A091C105B091C20585FDFF
:1026B00002C036952795253C49E03407B8F1409192
:1026C0000A0150E060E070E02CE1B695A79597957F
:1026D00087952A95D1F70097A105B10521F481E0EE
:1026E00090E0A0E0B0E084179507A607B707D8F4FC
:1026F00080910A018F3FB9F040E080910A014817AC
:1027000080F4842F90E0880F991FFC01E757FB4F5E
:1027100020813181FC01E55FFE4F318320834F5FD3
:10272000ECCF1092AA0410920A010BC02D3B82E05C
:10273000380720F080910A018031D8F08FEF809324
:102740000A01D0938804C0938704FF91EF91DF9131
:10275000CF91BF91AF919F918F917F916F915F9139
:102760004F913F912F911F910F900FBE0F901F908F
:10277000189510910A0181E0810F80930A01C90127
:102780000E942109E12FF0E0EE0FFF1FE757FB4FFA
:1027900091838083D6CF83E0809380008AE9809301
:1027A00081008091BF0586FD05C080918100806415
:1027B000809381008FEF9FEF909389008093880032
:1027C00080916F00806280936F0008950E94710D68
:1027D0008091D405843011F41092D40508956F309F
:1027E00018F086958058089589E0689F802D1124FF
:1027F0000895A0E0B0E0EFEFF3E10C946F2EC82F46
:102800000E94CC28009138041091390420913A0498
:1028100030913B046B017C01C01AD10AE20AF30A31
:102820009701860149E8C41643E1D406E104F104A6
:1028300010F010923C046093380470933904809334
:102840003A0490933B042091A9048FEF820F8230C9
:10285000D8F5E0913C04EE2309F44EC1E13011F4C7
:1028600082E0B8C1E03108F034C181E08E0F80937E
:102870003C04F0E0E757FB4FC083803109F0ACC166
:10288000EBE8F4E0213029F4A181A695A69580819A
:1028900008C080819181A92FA695A695A6959695A9
:1028A0008795A03148F4B0E090E0AA0FBB1FA55F68
:1028B000BE4F11969C938E931092AA04329684E098
:1028C000E939F807F9F688C1233009F005C1E0912C
:1028D0003C04E11104C0CF3009F07EC10DC1E831E4
:1028E00048F481E08E0F80933C04F0E0E857FB4F02
:1028F000C08372C1E83109F0ECC0C111EAC040E008
:1029000050E0ABE0CA01B3E0880F991FBA95E1F738
:10291000A49F9001A59F300D1124F901E757FB4FAB
:102920006081E1817E2F777075956795FC01EE0FD0
:10293000FF1FE55FFE4F71836083F901E657FB4F90
:10294000B081B695B695B695E181FE2FF295FF0F51
:10295000F07E6F2F6B2BE695E695E6957E2F7770D0
:1029600075956795FC01EE0FFF1FE35FFE4F7183C6
:102970006083F901E557FB4FB081B295B695B695E6
:10298000B370C181DC2FDD0FDD0F6D2F6B2BC29576
:10299000C695C695C370E281E170EE0FEE0F7E2FF3
:1029A0007C2B75956795FC01EE0FFF1FE15FFE4FD5
:1029B00071836083F901E357FB4FB081B695E181E4
:1029C000FE2FF795FF27F7956F2F6B2BE6957E2F40
:1029D000777075956795FC01EE0FFF1FEF5EFE4F58
:1029E00071836083F901E257FB4FB081B295BF70EC
:1029F000E181FE2FF295F07F6F2F6B2BE295EF7048
:102A00007E2F777075956795FC01EE0FFF1FED5EC9
:102A1000FE4F71836083F901E157FB4FB081BB1F0B
:102A2000BB27BB1FC181DC2FDD0F6D2F6B2BCC1F94
:102A3000CC27CC1FE281E370EE0F7E2F7C2B7595A7
:102A40006795FC01EE0FFF1FEB5EFE4F7183608305
:102A5000F901EF56FB4FB081B695B695E181FE2F97
:102A6000F295FF0FFF0FF07C6F2F6B2BE695E6952D
:102A70007E2F777075956795FC01EE0FFF1FE95E5D
:102A8000FE4F71836083F901EE56FB4F2081229542
:102A9000269527703181E32FEE0FEE0FEE0F6E2F8C
:102AA000622B732F72957695777075956795FC01FB
:102AB000EE0FFF1FE75EFE4F718360834F5F5F4F36
:102AC0004230510509F01ECF80919F0483FF109280
:102AD000AA0410923C0480C0243009F07DC06091AB
:102AE0003C0461110BC0C83AB1F410927505109204
:102AF000740588EA0E94610681E06CC0613019F4B7
:102B0000C093370404C0623031F4C09336048C2F74
:102B10000E9461065AC0E09136042E2F30E0220F49
:102B2000331F462F50E0C9010296841795073CF0E9
:102B3000633268F7FA01EA57FB4FC083E8CF2D5F95
:102B40003F4F8C2F90E0609174057091750542178E
:102B5000530749F4982F8827862797279093750560
:102B60008093740532C06817790769F5809137043E
:102B7000813049F5E13118F080E180933604F0901E
:102B80003604CAE8D4E000E010E00F15D0F4FE01EE
:102B90003197808190E0982F88272881822B63E0ED
:102BA000969587956A95E1F70E942109F801EE0F45
:102BB000FF1FE55FFE4F918380830F5F1F4F2296BB
:102BC000E4CF1092AA0410923C0480913C04882324
:102BD00019F08F5F80933C04CDB7DEB7E8E00C942A
:102BE0008B2EE82FF0E0E654FA4FE185E03150F407
:102BF000F894F0E0EE0FFF1FE55FFE4F80819181BA
:102C0000789408958EE08E0F8B3058F4F0E0E25FF8
:102C1000F10924E62E9FC0012F9F900D11240C96E0
:102C20000895E03FF1F028F4E03161F0E13161F026
:102C300006C0ED3F81F0EE3F89F0E13F49F080E0D2
:102C400092E0089582E101C083E10E940E2A089576
:102C500086E090E008958AEF93E008958FEF93E087
:102C6000089580E090E00895A2E2B0E0EAE3F6E1A2
:102C70000C94652E9E012F5F3F4F80E1D9011D927C
:102C80008A95E9F764E072E082EE95E029A33AA321
:102C90000E94B82A0E94BF0B1D8A1E8A1F8A188EA6
:102CA000312C212C00E0812C912C540170E4472E12
:102CB00071EE572E7DE9672E78E1772EE0E5CE2E76
:102CC000E3ECDE2EE12CF12C84EF91E0A0E0B0E00B
:102CD0008D8F9E8FAF8FB8A380EC91EDA8E9BBE1FB
:102CE000898F9A8FAB8FBC8F80E491EEADE9B8E10C
:102CF000898B9A8BAB8BBC8B82EE95E00E94CC2BA0
:102D0000892B09F4E1C082EE95E00E94F92B9C0129
:102D100033272C32310509F442C0ACF4233231059B
:102D200009F0ABC019821A821B821C821D821E828E
:102D30001F82188619861A861B861C861D861E868B
:102D40001F86188A60C02434310529F023353105E7
:102D500009F4B2C092C064E482EE95E00E948A2A2F
:102D60002AE030E040E451EE6DE978E182EE95E052
:102D70000E94182B6CE282EE95E00E948A2A2AE0DB
:102D800030E040EC51ED68E97BE182EE95E00E9495
:102D9000182B6CE282EE95E00E94CA2AADCF0F5F3D
:102DA000043009F0A9CF29813A814B815C81A8EEDA
:102DB000B3E00E94ED2D698B7A8B8B8B9C8B2D81E0
:102DC0003E814F8158850E94ED2D698F7A8F8B8FC0
:102DD0009C8F29853A854B855C852D8F3E8F4F8F43
:102DE00058A32D853E854F8558890E94ED2D6B0196
:102DF0007C0160323EE473078105910530F462E3A3
:102E00008CE10E94E20900E077CF603345E7740768
:102E10008105910510F462E2F3CF60345CE9750737
:102E20008105910510F466E2EBCF80E5C81683ECCE
:102E3000D806E104F10410F462E1E2CF90E6C9168D
:102E40009AEED906E104F10410F465E1D9CFA0E7C8
:102E5000CA16A1E1DA06A1E0EA06F10410F461E085
:102E6000CFCFB0EACB16B6E8DB06B1E0EB06F10453
:102E700010F463E0C5CF65E0C3CF10ED180F1A3032
:102E800008F03ACFE1E0F0E0EC0FFD1F24E0029FF4
:102E9000E00DF11D11242081318142815381AAE08E
:102EA000B0E00E94ED2D610F711D811D911D6083A9
:102EB00071838283938320CF49885A886B887C886A
:102EC000812C912C540118CF81149104A104B104D8
:102ED00089F4C301B2010E94510A61E070E080E010
:102EE00090E00E94EF281D8A1E8A1F8A188E312CBE
:102EF00022242A948D8D9E8DAF8DB8A188169906B7
:102F0000AA06BB06D0F40E940B0A2D893E894F8980
:102F1000588D280F311D411D511D2D8B3E8B4F8B20
:102F2000588F381608F4382E821508F4282E3FEFF3
:102F3000831A930AA30AB30A56C0C301B20128EE4A
:102F400033E040E050E00E94242EBA01A9012AE0BB
:102F500030E082EE95E00E946F2B6CE282EE95E00D
:102F60000E948A2A4AE050E0632D82EE95E00E949A
:102F70007E2B6CE282EE95E00E948A2A6D897E8922
:102F80008F89988DA50194010E94242EBA01A90170
:102F90002AE030E082EE95E00E946F2B6CE282EE38
:102FA00095E00E948A2A4AE050E0622D82EE95E088
:102FB0000E947E2B6CE282EE95E00E94CA2A4C0CA5
:102FC0005D1C6E1C7F1C898D9A8DAB8DBC8D84150C
:102FD0009505A605B70520F449885A886B887C8832
:102FE000812C912C540129893A894B895C89283E8E
:102FF00033404105510509F07FCEA296E2E10C94E1
:10300000812EACE1B0E0E7E0F8E10C946F2E0E9475
:10301000CC286B017C0181E00E94C10A14E703E027
:10302000198361E0CE0101960E941E0C0093730586
:103030000E949C0B6AEF70E080E090E00E94EF2815
:1030400080917305833089F482EE95E00E94CC2B49
:10305000892B59F40E94CC286C197D098E099F098F
:103060006038734C894C9140D8F28091730583305D
:1030700009F44FC08FE70E94BA090E94CD098983E5
:10308000843511F083E05CC00E94CD0910924605A2
:10309000809347050E94CD09209146053091470550
:1030A000280F311D30934705209346050E94CD0916
:1030B000809348050E94CD0980934905813110F71E
:1030C000F12C0F2D10E08091490590E0880F991F99
:1030D0000817190740F40E94CD09F801E65BFA4F82
:1030E0008083F394EECF80E7898361E0CE0101967F
:1030F0000E941E0C83E0809373050E949C0B62E388
:1031000070E080E090E00E94EF28809173058330AA
:1031100011F482E015C08FE70E94BA090E94CD0920
:103120008983803509F0AECF0FE915E00E94CD0903
:10313000F80181938F01F5E00A3B1F07B9F781E0A1
:103140006C96E8E00C948B2E80914505992787FDBD
:103150009095A92FB92FFC013196EB30F10508F0BD
:1031600066C0EC5CFF4F0C949C2E62E778E082EE28
:1031700095E00E94A62A84E893E00E94730C6AE519
:1031800078E082EE95E00E94A62A65E378E082EE80
:1031900095E00E94A62A6BE078E082EE95E00E941E
:1031A000A62A6AEE77E082EE95E00E94A62A6DEBF1
:1031B00077E082EE95E00E94A62A67E977E082EE4A
:1031C00095E00E94A62A63E777E082EE95E00E94F0
:1031D000A62A6CE477E082EE95E00E94A62A82EEB1
:1031E00095E00E94922A0E94B10D21C06FE277E023
:1031F0001AC06AE077E017C065EF76E014C066EDAC
:1032000076E011C062E976E00EC06DE776E00BC0B3
:1032100068E676E082EE95E00E94A62A62E276E019
:1032200002C06CE076E082EE95E00E94A62A6AE099
:1032300070E080E090E00E94EF2882EE95E00E942E
:10324000CC2B892B29F082EE95E00E94F92BF5CF4B
:103250000895ACE1B0E0EFE2F9E10C946F2E9091AB
:1032600045059F3F09F023C1482F50E0FA013A97E6
:10327000EF36F10508F00FC1E15CFF4F0C949C2E76
:1032800061E172E0A0C06DE172E082EE95E00E9423
:10329000B82A85E789838BE1EFE9F5E0DE01129634
:1032A00001900D928A95E1F76CE1CE0101960E94A2
:1032B0001E0C0E949C0B83E08093730568EC70E009
:1032C00080E090E00E94EF2880917305843009F03F
:1032D000E2C08FE70E94BA090E94CD098983853533
:1032E00009F0D9C06DEE74E082EE95E00E94A62A46
:1032F0006FEC74E082EE95E00E94A62A61EB74E028
:1033000096C065E372E082EE95E00E94B82A89E6F5
:10331000898361E0CE0101960E941E0C0E949C0BE5
:1033200083E08093730568EC70E080E090E00E9499
:10333000EF2880917305843009F0ADC08FE70E94BB
:10334000BA090E94CD0989838E010E5F1F4F7E014D
:103350004DE1E40EF11C0E94CD09F80181938F012B
:10336000EE15FF05C1F78BE1FE013296AFE9B5E03E
:1033700001900D928A95E1F78981893409F08BC01B
:1033800063E974E082EE95E00E94A62A65E774E0A6
:1033900082EE95E00E94A62A67E574E048C06FE4DB
:1033A00072E082EE95E00E94B82A8EEF8093450588
:1033B00072C080528750805390914805981708F04A
:1033C00066C06EE572E082EE95E00E94B82A63C0A6
:1033D00084E18093450560E274E029C085E1809333
:1033E000450569EE73E023C086E18093450562EBF5
:1033F00073E01DC087E18093450568E673E017C060
:1034000088E18093450567E573E011C089E1809309
:10341000450563E473E00BC08AE1809345056EE2E5
:1034200073E005C08BE18093450566E073E082EEB2
:1034300095E00E94A62A2FC06CEE72E082EE95E025
:103440000E94A62A8091AD0591E01DC066ED72E054
:1034500082EE95E00E94A62A8091AD0592E013C00D
:1034600061EC72E082EE95E00E94A62A8091AD05A3
:1034700094E009C066EA72E082EE95E00E94A62A16
:103480008091AD0598E089278093AD058FEF8093FB
:1034900045050E94521082EE95E00E94CC2B892BAC
:1034A00009F45BC182EE95E00E94F92BF4CF0E94F3
:1034B0005111882309F451C18091DF04811104C0A6
:1034C0008FEF8093450541C140E050E060E070E03F
:1034D00080EE94E00E94132F40914505042F1127A0
:1034E00007FD1095212F312FF8013197EB31F105B0
:1034F00008F01BC1E255FF4F0C949C2E552747FD49
:1035000050952091480530E0241735070CF40DC183
:103510008B019C010150110921093109003211056B
:103520002105310558F0C0904905EBE4F5E0F12C98
:10353000D12CA8E2EA2E415051090FC0FA01E15600
:10354000FA4F61506083D9C0DF0111972C9130E0B0
:103550002417350729F0F3943296FC10F5CFCBC031
:103560000E2D10E020E030E0061717072807390776
:1035700041F42081DA01A156BA4F11962C93DD2433
:10358000D394E394E8CF6F3F71058105910511F065
:1035900008F0CBC06093B705B0C06F3F71058105DF
:1035A000910511F008F0C1C06093B805A6C06F3F47
:1035B00071058105910511F008F0B7C06093B90558
:1035C0009CC02091E00420622037E9F440E050E004
:1035D00060E070E081EE94E00E94132F9B01AC014B
:1035E000DC01CB010197A109B1090897A105B1053B
:1035F00008F0AEC0A4EDB0E30E94ED2D6A5E7C4AF7
:103600008A46954E24C02636E9F440E050E060E05A
:1036100070E081EE94E00E94132F9B01AC01DC016D
:10362000CB010197A109B1090797A105B10508F0E0
:103630008FC0A8EAB1E60E94ED2D645E7C438E4601
:10364000944E05C0611571058105910579F08B01D6
:103650009C010054114E2D4938410138F0EF1F07ED
:10366000FAEF2F07F2E03F0708F05FC06093AF0565
:103670007093B0058093B1059093B2053EC06F3F43
:1036800071058105910511F008F04FC06093B305F5
:1036900034C08B019C0101501109210931090F3FF0
:1036A00011052105310508F040C06093B40525C01F
:1036B0008B019C01045C1940210931090D344DE155
:1036C00014072105310528F47093B6056093B505FC
:1036D00014C0611571058105910521F48FEF809368
:1036E000AE050BC06134710581059105F0F46150A0
:1036F0006093AE0502C0DD20C1F08091DE0481112F
:103700001AC080917F0590918005A0918105B091AC
:1037100082050196A11DB11D80937F0590938005C0
:10372000A0938105B093820506C060E772E082EE47
:1037300095E00E94B82A0E9447118FEF80934505BB
:103740006AE082EE95E00E94CA2A0E94521005C0EB
:1037500061E070E080E090E07ACF6C96E8E00C9455
:103760008B2E6AE572E082EE95E00E94A62A62E462
:1037700072E082EE95E00E94A62A82EE95E00E9419
:10378000CC2B892B31F082EE95E00E94F92B0E9420
:1037900029190E940118823029F0833051F46DE01C
:1037A00072E002C064E272E082EE95E00E94A62A16
:1037B00008958FEF809345051092DE040E94521009
:1037C000809145058E3F69F082EE95E00E94CC2BFA
:1037D000892BB1F382EE95E00E94F92B0E94291902
:1037E000EFCF08950F931F93109145051F3F09F0E8
:1037F000D2C0893409F457C000F5883309F469C090
:1038000058F4803309F477C008F061C08B3109F4B3
:1038100040C08132B1F1B9C0813409F487C030F4BD
:10382000893309F466C0803461F1AFC0823409F491
:103830008EC0863409F448C0A8C0823609F487C017
:1038400078F4883531F128F48235C1F18335E1F01F
:103850009CC08A3509F494C0813609F467C095C0CC
:10386000823761F128F4863679F18936E1F08DC02E
:10387000883779F08A3709F483C0833709F085C027
:1038800003C061E172E015C00E94820D6EE872E033
:1038900004C00E948B0D68EA72E082EE95E00E94FF
:1038A000B82A8EEF70C00E947A060E94BF0667ECAD
:1038B00072E082EE95E00E94B82A67C081E00E9423
:1038C000DF0660EE72E0F5CF0E94FC105EC0805310
:1038D0005AC06AEF71E082EE95E00E94A62A9091AC
:1038E0009E0588E0890F8871977E892B80939E05BD
:1038F0001AC089E048C067EE71E082EE95E00E9450
:10390000A62A8091BF059091C005A091C105B091F4
:10391000C20520E182278093BF059093C005A09344
:10392000C105B093C205109345052FC061ED71E04C
:1039300082EE95E00E94A62A8091BF059091C00575
:10394000A091C105B091C20540E4842710C060EC8D
:1039500071E082EE95E00E94A62A8091BF059091C9
:10396000C005A091C105B091C20520E282278093D5
:10397000BF059093C005A093C105B093C20502C0D6
:103980000E94B11B8FEF80934505809145058E3FC6
:1039900009F0D4C0DDC00E945111882309F4D8C0B9
:1039A0008091DF04811104C08FEF80934505C6C06C
:1039B00040E050E060E070E080EE94E00E94132F61
:1039C00000914505112707FD1095212F312FF80192
:1039D0003197E930F10508F0B4C0E753FF4F0C947C
:1039E0009C2E8B019C010154114E2D4938410F37FB
:1039F000104F2A4F324008F0A4C060937B057093AB
:103A00007C0580937D0590937E0577C060937F054C
:103A100070938005809381059093820581E0809367
:103A2000DE046BC0683071058105910508F089C01E
:103A30006093830562C08B019C010150110921092B
:103A400031090A3011052105310508F07AC060936B
:103A5000840553C061EB71E080EE94E00E944D302C
:103A600010E0009799F00E942730009779F0183104
:103A700030F4E12FF0E0EA58FA4F87871F5F61EBDF
:103A800071E080E090E00E944D30EBCF1831A8F556
:103A9000E12FF0E0EA58FA4F17861F5FF7CF653045
:103AA00071058105910508F04CC060939D0525C006
:103AB0008B019C01015011092109310906301105C2
:103AC00021053105F0F520919E05287F262B2093B6
:103AD0009E0513C08B019C01015011092109310978
:103AE0000115124C2140310560F560937705709304
:103AF00078058093790590937A058091DE04811191
:103B000013C080917F0590918005A0918105B091AF
:103B100082050196A11DB11D80937F0590938005BC
:103B2000A0938105B09382050E9447118FEF809387
:103B300045056AE082EE95E00E94CA2A0E94A41818
:103B400007C060E772E082EE95E00E94B82AECCFF1
:103B50001F910F9108958FEF809345051092DE0419
:103B60000E94A418809145058E3F69F082EE95E091
:103B70000E94CC2B892BB1F382EE95E00E94F92BA9
:103B80000E94F21BEFCF6AE070E080E090E00E94BC
:103B9000EF2882EE95E00E94CC2B892B29F082EE53
:103BA00095E00E94F92BF5CF0895CF93C82F682F89
:103BB00082EE95E00E94262C90916A059C279093B6
:103BC0006A05CF910895A1E0B0E0E9EEFDE10C9423
:103BD000752E99830E94D51D9981892F0E94D51D2C
:103BE0002196E2E00C94912E1F93CF93DF93182F30
:103BF000EB0110926A0565EB70E082EE95E00E94A1
:103C0000590662E670E082EE95E00E945906812F27
:103C10000E94D51DCE010E94E31DDF91CF911F911F
:103C2000089560916A0582EE95E00E94262C089521
:103C3000A1E2B0E0EEE1FEE10C94712E7B018A017D
:103C40008C3009F452C108F040C0863009F4BCC081
:103C500018F5833009F491C070F4813009F472C012
:103C6000823009F047C26BE170E082E00E94F41DEF
:103C70000FE915E078C0843009F487C0853009F079
:103C800039C26091490570E0660F771F85E00E9498
:103C9000F41D0AE415E086C0893009F4A7C070F469
:103CA000873009F49BC0883009F024C261E070E0DD
:103CB00088E00E94F41D8091D40522C28A3009F464
:103CC000CAC08B3009F4F1C015C28A3609F474C138
:103CD000D8F4873609F439C138F4853609F40DC1B2
:103CE000863609F41EC106C2883609F436C1893603
:103CF00009F000C261E070E089E60E94F41D0E94B4
:103D00007A060E94BF06F4C18D3609F4D3C138F497
:103D10008B3609F490C18C3609F499C1EBC18E360B
:103D200009F4DBC1873C09F0E5C161E070E087EC94
:103D30000E94F41D81E00E94D51D0E94111E109268
:103D40006B05E2C169E270E081E00E94F41D06E7C4
:103D500015E0F80181918F010E94D51DF5E00F3922
:103D60001F07B9F7CFC1F80181918F010E94D51DBE
:103D7000F5E00A3B1F07B9F7C5C161E070E083E0D9
:103D80000E94F41D0E940118BBC161E070E084E054
:103D90000E94F41D81E00E94D51D0E94111E0E9408
:103DA0003416B2C18091490590E0880F991F98019F
:103DB0002A5435402817390708F0A4C1F801819129
:103DC0008F010E94D51DEECF62E070E086E00E9478
:103DD000F41D84E893E00E94E31D94C161E070E06B
:103DE00087E00E94F41D809148058AC186E6898398
:103DF00061E0CE0101960E941E0C0E949C0B83E0A4
:103E00008093730568EC70E080E090E00E94EF28FA
:103E1000809173058430D9F48FE70E94BA090E941B
:103E2000CD098983863469F460E270E089E00E94FC
:103E3000F41D10E20E94CD090E94D51D1150D1F74A
:103E400061C161E070E089E00E94F41D51C161E050
:103E500070E089E052C169E170E08AE00E94F41DDF
:103E60001092BA05209172058091BF059091C0050E
:103E7000A091C105B091C205222311F0806801C054
:103E80008F778093BF059093C005A093C105B09331
:103E9000C2050AEB15E0F80181918F010E94D51D42
:103EA000F5E0033D1F07B9F72DC161E270E08BE03B
:103EB0000E94F41D8091AA048F3F39F08091AA04DA
:103EC00091E0980F9093AA0402C08091AA040E94E6
:103ED000D51D10E0812F0E94F1150E944C090E940F
:103EE000E31D1F5F1031B1F70DC161E070E08CE0A0
:103EF0000E94F41D8091D30503C161E070E085E666
:103F00000E94F41D89E2E816F10409F0F8C0D80116
:103F1000E6E7F5E08D91819385E0EF39F807D1F779
:103F2000E7C061E070E086E60E94F41DEBE1EE166A
:103F3000F10409F0E4C0D801EFE9F5E08D91819337
:103F400085E0EA3BF807D1F7D3C061E070E087E68F
:103F50000E94F41D0E94820DCBC061E070E088E6F3
:103F60000E94F41D85E789838BE1EFE9F5E0DE012E
:103F7000129601900D928A95E1F76CE1CE010196BF
:103F80000E941E0C0E949C0B83E08093730560E2EC
:103F900073E080E090E00E94EF2880917305843008
:103FA00009F0ADC08FE70E94BA090E94CD0989834C
:103FB000853509F0A4C09CC061E070E08AE60E94EB
:103FC000F41D89E6898361E0CE0101960E941E0CF2
:103FD0000E949C0B83E08093730560E273E080E0B5
:103FE00090E00E94EF2880917305843009F087C02B
:103FF0008FE70E94BA090E94CD0989838E010E5F66
:104000001F4F7E01EDE1EE0EF11C0E94CD09F8017B
:1040100081938F01EE15FF05C1F78BE1FE0132960A
:10402000AFE9B5E001900D928A95E1F78981893475
:1040300009F065C05DC061E070E08BE60E94F41D90
:10404000F80180818093D4050E948B0D51C061E0FE
:1040500070E08CE60E94F41DF0E2EF16F10461F4CA
:1040600087E6898380E2F801DE01129601900D92C5
:104070008A95E1F761E203C087E4898361E0CE01BC
:1040800001960E941E0C0E949C0B83E08093730596
:104090006CE474E080E090E00E94EF28809173056A
:1040A000843069F58FE70E94BA090E94CD098734F0
:1040B00031F51EC061E070E08DE60E94F41D89E1DB
:1040C000E816F104E1F4D801EAEBF5E08D91819373
:1040D00085E0E33DF807D1F70BC061E070E08EE6C4
:1040E0000E94F41DF80180818093D3050E946C0D1D
:1040F00081E006C061E070E08AEC0E94F41D80E07F
:104100000E94D51D0E94111EA196E6E00C948D2EF2
:10411000A0E0B0E0EEE8F0E20C946F2ECAECD3E041
:1041200014E606E035E0F32E44E0E42E53E0D52E0D
:1041300062E0C62E82EE95E00E94CC2B892B09F41A
:104140009BC082EE95E00E94F92B282F80933504C6
:104150004091340450E04730510560F7FA01EE52C7
:10416000FF4F0C949C2E853B29F781E0809334040B
:10417000E1CF823609F07DC0C0923404DBCF80935A
:10418000330480933204D0923404D4CF9C0133277B
:104190003093310420933004909132049827909307
:1041A0003204E0923404C6CF382F222740913004E5
:1041B00050913104242B352B30933104209330045B
:1041C00090913204982790933204F092340425366B
:1041D000310508F4AFCF61E070E08CEC0E94F41D73
:1041E00081E00E94D51D0E94111E43C020912E0423
:1041F00030912F04F901E653FC4F808390913204F3
:10420000982790933204C901019690932F048093CC
:104210002E0420913004309131048217930708F462
:1042200089CF0093340486CF8091320482130BC06F
:1042300060912E0470912F044AEC53E08091330476
:104240000E94181E0DC062E070E08BEC0E94F41D0D
:10425000809133040E94D51D80916A050E94D51D6E
:10426000FE01812F11928A95E9F710922F04109286
:104270002E04109234045ECFCDB7DEB7E8E00C9484
:104280008B2E81E080936B0580916B05882349F02C
:1042900082EE95E00E94CC2B892BB1F30E948820FE
:1042A000F3CF0895AAE2B0E0E8E5F1E20C946D2EB8
:1042B0000E94C0286B017C0181E00E94C10A82EE4D
:1042C00095E00E94CC2B892B29F082EE95E00E948C
:1042D000F92BF5CF439811E072E6B72EE9E2AE2E46
:1042E00003E00E94C0286C197D098E099F09693C72
:1042F000710581059105D0F11123C1F10E94C028FB
:104300006B017C01429A80ED97E00E94B607B9826A
:10431000E6E7F5E0DE0112968A2D01900D928A956E
:10432000E1F76AE2CE0101960E941E0C429880E0FD
:1043300090E00E94B607009373050E949C0B62E315
:1043400070E080E090E00E94EF2880917305843057
:1043500061F4009373058FE70E94BA090E94CD09AA
:1043600011E0823419F410E001C011E082E10E94F2
:10437000E529892B81F411E00EC0439A429A82EE1E
:1043800095E00E94F92B8D309105A9F05CF40A9715
:1043900091F04398429882EE95E00E94CC2B892BB5
:1043A00061F79FCF8332910579F08234910589F7C7
:1043B0000E944121EECF62EB71E082EE95E00E9417
:1043C000A62A0E94AB1DE5CF0E943416E2CF8F9241
:1043D0009F92AF92BF92CF92DF92EF92FF921F9384
:1043E000CF93DF9382E10E94E529892B09F089C0F0
:1043F00068EC70E080E090E00E94EF2880E090E0C0
:104400000E94B6070E94C0284B015C016B017C0131
:1044100080ECC80E82E1D81EE11CF11C0E94C0286D
:104420006C157D058E059F0530F482E10E94E5291B
:10443000892BA1F364C082E10E94E529892B09F050
:104440005EC080ED97E00E94B6070E94C0286B0115
:104450007C01D0E0C1E088E4880E86E2981EA11CB1
:10446000B11C11E082E10E94E529892B21F58C1411
:104470009D04AE04BF0430F480ED97E00E94B607BF
:10448000D1E0F0CF0E94C0286C197D098E099F09E8
:10449000693C71058105910528F30E94C0286B01D4
:1044A0007C01C12719F080ED97E002C080E090E028
:1044B0000E94B607D7CF80E090E00E94B607DD23C8
:1044C000B9F08091D30590E0019665E070E00E941C
:1044D000102E8093D3050E946C0D0E94E6130E945B
:1044E0008B0D64EF71E080E090E00E94EF2809C03E
:1044F00080E00E94DF060E9403120E94820D0E944B
:104500005221DF91CF911F91FF90EF90DF90CF90DC
:10451000BF90AF909F908F900895CF92DF92EF92CF
:10452000FF9280E00E941D080E94F40761E081E193
:104530000E94792961E080E10E94792960E082E1AE
:104540000E94792960E088E00E94792961E088E092
:104550000E94B2290E949F0740E052EC61E070E0A7
:1045600082EE95E00E94142D0E94E6130E948B0DAE
:104570000E94CB138FEF8093AA040E9409087894BD
:104580000E94C0286B017C018091AA048F3F59F4DE
:104590000E94C0286C197D098E099F09603D7740F3
:1045A0008105910588F380ED97E00E94B60761E0F0
:1045B00082E10E94B229439A82EE95E00E94CC2BC0
:1045C000892B29F082EE95E00E94F92BF5CF6DEF53
:1045D00072E082EE95E00E94872A84E893E00E94D0
:1045E000730C64E173E082EE95E00E94872A4AE052
:1045F00050E068E070E082EE95E00E94572B62E3A5
:1046000070E080E090E00E94EF2882EE95E00E944A
:10461000CC2B04970CF182EE95E00E94F92B8234AA
:104620009105D1F482EE95E00E94F92B8E3491052C
:1046300099F482EE95E00E94F92B8434910561F49F
:1046400082EE95E00E94F92B819731F480E090E0B2
:104650000E94B6070E94522140917705509178053B
:104660006091790570917A05DB01CA010197A10972
:10467000B1090497A105B10568F44093A90443303A
:1046800029F440EA56E861E070E004C040E052ECF2
:1046900061E070E082EE95E00E94142D0E94E72117
:1046A000439880E090E00E94B6070E94CB131092DE
:1046B000C5048091BF0583FF11C080918B058823BD
:1046C00051F080919205882331F0809199058823DB
:1046D00011F087E001C085E08093C50480E00E946E
:1046E000C10A8091C6040E94F5090E949C0B109299
:1046F0003F0410923E0410923D04F12C8091D405A9
:104700008F15B0F062E370E080E090E00E94EF2847
:1047100080ED97E00E94B60762E370E080E090E0F1
:104720000E94EF2880E090E00E94B607F394E6CF65
:1047300080919E0584FF08C0982F987181E0983180
:1047400009F080E00E94BF118FE00E941D08FF90D9
:10475000EF90DF90CF900895EF92FF920F931F9309
:10476000CF93DF938C016EE770E082EE95E00E94BC
:104770005906E801F12CF0E2EF2E8E0188818D5769
:10478000823048F46DE770E082EE95E00E945906B1
:1047900088818E2588832196F801608182EE95E0DC
:1047A0000E94262CF394F9E0FF12E7CF6EE770E049
:1047B00082EE95E00E945906CDB7DEB7E6E00C9494
:1047C0008D2EA9E0B0E0E7EEF3E20C94752E909107
:1047D000C70491110EC09EEF99838A836B8350E0CA
:1047E000559547954C832D83198618861F821E8206
:1047F0002EC04091CC04842F90E0B4E0959587952D
:10480000BA95E1F7242F2F7030E08217930719F142
:104810008DEF89831B82FE01349650E0842F90E057
:10482000A4E095958795AA95E1F7242F2F7030E0A5
:104830008217930749F0DC01A353BB4F8C918193FE
:10484000405F5F5F563051F74093CC045A83CE01EE
:1048500001960E94AC238091C70490E0019666E027
:1048600070E00E94102E8093C7042996E2E00C9419
:10487000912EA0E0B0E0EFE3F4E20C946E2E6C0118
:104880006EE770E082EE95E00E9459068601E12C09
:10489000F12CC0E0D0E030E2B32EF801608183E873
:1048A000860F823078F46DE770E082EE95E00E942A
:1048B0005906F80160816B2570E082EE95E00E9458
:1048C000590604C082EE95E00E94262CE114F10402
:1048D00059F0F80180819E01280F311DC901C92FAF
:1048E000DD27C80FD91FDD273FEFE31AF30A89E060
:1048F000E816F10459F028E0E216F10421F48C2FB7
:104900008095F60180870F5F1F4FC7CFCDB7DEB709
:10491000E9E00C948A2EA9E0B0E0E1E9F4E20C941D
:10492000752EE82F362F8091C70490E0019664E23F
:1049300070E00E94102E8093C70458E9598350E11B
:104940005A83813089F048F08230B9F08330D9F44D
:104950008B8381EF8C833D8319C085E08B8381EF4E
:104960008C832F5F2D8312C08B8381EF8C8384E631
:10497000489FA00111245D8309C084E08B8381EFEF
:104980008C83ED8303C00E94FC1104C0CE0101960C
:104990000E9439242996E2E00C94912EA2E0B0E026
:1049A000E4EDF4E20C946A2E182F762E2A834983C4
:1049B0000E94CC286B017C018091DD048090C804AA
:1049C0009090C904A090CA04B090CB042A81498178
:1049D0008823C1F0D701C60188199909AA09BB0922
:1049E0004C015D0191EE89169EE29906A104B10485
:1049F00020F1241708F4422F202F672D812F0E94C9
:104A00008B2413C0D701C60188199909AA09BB09CB
:104A10004C015D0191E3891695E79906A104B10463
:104A200060F0672D812F0E94E123C092C804D092CC
:104A3000C904E092CA04F092CB042296EDE00C94F3
:104A4000862EA2E2B0E0E7E2F5E20C946B2E8CE059
:104A50000E94DC0981110DC06CE173E082EE95E0EB
:104A60000E94B82A439A80E00E94C10A0E949C0BCF
:104A7000439882EE95E00E94CC2B892B01F182EEC7
:104A800095E00E94F92B9091A904992319F00E94B6
:104A9000F913EFCF40913E0450E09A012F5F3F4F52
:104AA0002F71332760913F0470E02617370709F311
:104AB000FA01E75BFB4F808320933E04DACF8091BD
:104AC0007305843009F086C00E94CC2861157105F9
:104AD0008105910549F06093B7047093B804809301
:104AE000B9049093BA040CC081E090E0A0E0B0E07B
:104AF0008093B7049093B804A093B904B093BA0418
:104B00008091AD049091AE0481609093AE04809347
:104B1000AD0483E0809373058FE70E94BA0909E62C
:104B200014E00E94CD09F80181938F01F4E002376F
:104B30001F07B9F72091720480916904982F92277A
:104B400096FF3BC090E4922790937204982F98733D
:104B50009833F1F410E0212F30E0809169048770E0
:104B600090E0821793074CF11F5F20919E05812FE3
:104B700090E0FC01E759FB4F24FF04C080810E94B4
:104B8000DE11E9CF608182EE95E00E94262CE3CF12
:104B90008F7399F480916A048093B60480916B04BA
:104BA0008093B40480916C048093B30480916F046B
:104BB00090E09093AC048093AB0480913D048130ED
:104BC00019F482E080933D0480913D04833011F418
:104BD00010923D040E94CC286B017C018091AF04AF
:104BE0009091B004A091B104B091B2040097A105D6
:104BF000B105C9F0A7019601281B390B4A0B5B0BC5
:104C0000DA01C901883B9B40A105B10560F00E9413
:104C10000B0A8093B5041092AF041092B004109266
:104C2000B1041092B2048091BB049091BC04A09195
:104C3000BD04B091BE0446015701881A990AAA0A18
:104C4000BB0A86E795E00E94370886169706A806F5
:104C5000B90608F4A8C0C092BB04D092BC04E0928C
:104C6000BD04F092BE040E9457068091AA048830C9
:104C7000A0F08091BF059091C005A091C105B091B1
:104C8000C2055CE1B695A795979587955A95D1F79A
:104C9000892B8A2B8B2B09F09EC18091AA048F5FF0
:104CA0008093AA048091B7049091B804A091B904AC
:104CB000B091BA040097A105B105F1F0C81AD90A5C
:104CC000EA0AFB0A86E795E00E9437086C157D0525
:104CD0008E059F0508F006C18091BF0584FD04C0C4
:104CE00080ED97E00E94B6071092B7041092B804C6
:104CF0001092B9041092BA0490917204907C90932F
:104D0000720450913E0480913F0420913D04581755
:104D100009F405C1223009F002C190589093720441
:104D2000E0919E05E770F0E0E658FC4F6081693045
:104D300008F0DDC0615040E04613DBC080933F04C3
:104D400087E3840F90917204892B809372044093BF
:104D5000400483E080933D04429A809183059091C2
:104D6000C504911129C10E94BC0A8091C6040E9409
:104D7000F509E0919E05E770F0E0E658FC4F608190
:104D800082E794E00E94D70BE091C604EF5FE093C6
:104D9000C604E83109F41CC1F0E0EA58FA4F8785EF
:104DA000882309F415C10E94460C813069F5809171
:104DB0009E05887149F18091AD049091AE04880FF1
:104DC000991F9093AE048093AD0483E080937305A4
:104DD0000E949C0B0E94CC286093AF047093B00497
:104DE0008093B1049093B204672B682B692B61F414
:104DF00081E090E0A0E0B0E08093AF049093B00435
:104E0000A093B104B093B20480919E0584FF1FC0AB
:104E10008091AD049091AE048E7F0E946D09182F91
:104E20006091AB048091B6040E94EF13482F612F6C
:104E30008091B50449A30E94EF130091D405282F57
:104E400049A16091B3048091B4040E94CE24429899
:104E50008091C3048130C1F018F08230B1F1C8C034
:104E600082E10E94E529892B09F0C2C081E080938C
:104E7000C3040E94C0286093BF047093C004809351
:104E8000C1049093C204B4C082E10E94E529892B39
:104E900031F50E94C028C090BF04D090C004E090BB
:104EA000C104F090C2046C197D098E099F09693E06
:104EB00073408105910508F49BC082E08093C30490
:104EC00080ED97E00E94B60793C082E10E94E52939
:104ED000892B09F48DC080E090E00E94B607109203
:104EE000C30486C080E090E00E94B60705CF68E06A
:104EF00022CF851709F422CF4F5F242F30E090E0B6
:104F0000F901EE58FB4FDC01A75BBB4F7C9170832E
:104F1000F901E05CFB4F708301968F710DCF243057
:104F2000B1F42091400481E494E0A3E7B4E0FC01F3
:104F30003E2F381B321718F431913D93F9CF87E398
:104F4000820F90917204892B8093720402CF80911A
:104F5000C304823051F4916090937204439A8E019D
:104F60000F5F1F4FF12CB80110C0439880913D0492
:104F7000811103C081E080933D0480913D04833022
:104F800071F784E080933D04EACF8F2D69A37AA363
:104F90000E94F115F801819391938F01F39469A117
:104FA0007AA1F0E1FF12F1CF80919E0543E754E032
:104FB00087700E94BC08D0CE882309F4D4CE2091FB
:104FC000C40431E0320F3093C4042913CCCE0CC09A
:104FD0001092C604E8CE8091AA04883009F4439A5E
:104FE00089E08093AA04DFCE1092C4048150BBCE26
:104FF000A296ECE00C94872E8230E8F4E82FF0E0E3
:10500000EE0FFF1FEB52FA4F71836083813041F046
:10501000809169008C7F842B80936900E89A0895C1
:1050200080916900440F551F440F551F837F842BC7
:1050300080936900E99A08951F920F920FB60F921C
:1050400011242F933F934F935F936F937F938F938D
:105050009F93AF93BF93EF93FF938091D50590916A
:10506000D605892B29F0E091D505F091D605099553
:10507000FF91EF91BF91AF919F918F917F916F9130
:105080005F914F913F912F910F900FBE0F901F9006
:1050900018951F920F920FB60F9211242F933F93E2
:1050A0004F935F936F937F938F939F93AF93BF9330
:1050B000EF93FF938091D7059091D805892B29F024
:1050C000E091D705F091D8050995FF91EF91BF9137
:1050D000AF919F918F917F916F915F914F913F9190
:1050E0002F910F900FBE0F901F9018951F920F9247
:1050F0000FB60F9211242F933F938F939F93AF93EB
:10510000BF938091DA059091DB05A091DC05B09109
:10511000DD053091D90523E0230F2D3720F40196CA
:10512000A11DB11D05C026E8230F0296A11DB11DCA
:105130002093D9058093DA059093DB05A093DC05D5
:10514000B093DD058091DE059091DF05A091E0052B
:10515000B091E1050196A11DB11D8093DE059093EC
:10516000DF05A093E005B093E105BF91AF919F915A
:105170008F913F912F910F900FBE0F901F90189518
:105180002FB7F8946091DA057091DB058091DC050A
:105190009091DD052FBF08953FB7F8948091DE050B
:1051A0009091DF05A091E005B091E10526B5A89B9F
:1051B00005C02F3F19F00196A11DB11D3FBF662705
:1051C000782F892F9A2F620F711D811D911D42E04A
:1051D000660F771F881F991F4A95D1F70895CF92C0
:1051E000DF92EF92FF92CF93DF936B017C010E94DD
:1051F000CC28EB01C114D104E104F10479F00E9440
:10520000CC286C1B7D0B683E7340A0F381E0C81A6C
:10521000D108E108F108C851DC4FECCFDF91CF9104
:10522000FF90EF90DF90CF900895789484B58260DE
:1052300084BD84B5816084BD85B5826085BD85B53A
:10524000816085BDEEE6F0E0808181608083E1E8E9
:10525000F0E0108280818260808380818160808321
:10526000E0E8F0E0808181608083E1EBF0E0808124
:1052700084608083E0EBF0E0808181608083EAE7F6
:10528000F0E080818460808380818260808380817F
:10529000816080838081806880831092C10008953E
:1052A000833081F028F4813099F08230A1F00895A4
:1052B0008630A9F08730B9F08430D1F48091800035
:1052C0008F7D03C0809180008F7780938000089548
:1052D00084B58F7702C084B58F7D84BD0895809199
:1052E000B0008F7703C08091B0008F7D8093B000B5
:1052F0000895CF93DF9390E0FC01ED50F44F24919B
:10530000FC01E95FF34F8491882349F190E0880F15
:10531000991FFC01E15DF34FA591B4918B5D934F13
:10532000FC01C591D4919FB7611108C0F8948C918C
:10533000209582238C93888182230AC0623051F4A5
:10534000F8948C91322F309583238C938881822B13
:10535000888304C0F8948C91822B8C939FBFDF913B
:10536000CF910895A1E0B0E0E8EBF9E20C94732E40
:10537000282F30E0F901E152F44F8491F901ED500A
:10538000F44F1491F901E95FF34F04910023C9F040
:10539000882321F069830E9450296981E02FF0E081
:1053A000EE0FFF1FEB5DF34FA591B4919FB7F894FB
:1053B0008C91611103C01095812301C0812B8C93C6
:1053C0009FBF2196E4E00C948F2ECF93DF93282F7C
:1053D00030E0F901E152F44F8491F901ED50F44FBE
:1053E000D491F901E95FF34FC491CC2391F081117D
:1053F0000E945029EC2FF0E0EE0FFF1FE55EF34F07
:10540000A591B4912C912D2381E090E021F480E0CE
:1054100002C080E090E0DF91CF9108958E3008F0D7
:105420008E50877020919D0190E4299F9001112456
:10543000822B80937C0080917A00806480937A0034
:1054400080917A0086FDFCCF8091780020917900D0
:1054500090E0922B0895A0E0B0E0E1E3FAE20C9432
:105460006F2E6C017A01EB01E60EF71E00E010E0F2
:10547000CE15DF0561F06991D601ED91FC910190A7
:10548000F081E02DC6010995080F191FF1CFC80161
:10549000CDB7DEB7E8E00C948B2E6115710589F06D
:1054A000DB010D900020E9F7AD0141505109461B89
:1054B000570BDC01ED91FC910280F381E02D099501
:1054C000089580E090E00895EF92FF920F931F936C
:1054D000CF93DF938C01FB01C0E0D0E064917F01AA
:1054E0008FEFE81AF80A662361F0D801ED91FC917C
:1054F0000190F081E02DC8010995C80FD91FF7016F
:10550000EDCFCE01CDB7DEB7E6E00C948D2E0E9434
:105510004D2A0895DC01ED91FC910190F081E02D80
:10552000099508950F931F93CF93DF93EC016DE0DE
:105530000E948A2A8C016AE0CE010E948A2A800F8A
:10554000911FDF91CF911F910F9108950F931F939A
:10555000CF93DF93EC010E94642A8C01CE010E945C
:10556000922A800F911FDF91CF911F910F91089583
:105570000F931F93CF93DF93EC010E944D2A8C0170
:10558000CE010E94922A800F911FDF91CF911F912F
:105590000F9108950F931F93CF93DF93EC010E9417
:1055A0008A2A8C01CE010E94922A800F911FDF91DE
:1055B000CF911F910F910895A1E2B0E0E2EEFAE2DF
:1055C0000C946B2E7C01C42EE52FCB01D22E19A298
:1055D00021E02D1510F02AE0D22E8E010F5D1F4F15
:1055E0008D2C912CA12CB12C6C2D7E2FA50194011A
:1055F0000E94242E8C2DD29E801911240150110955
:105600008A3010F4805D01C0895CF8018083211527
:1056100031054105510521F0C22EE32FCA01E4CF27
:10562000B801C7010E944D2AA196ECE00C94872E88
:10563000A0E0B0E0EEE1FBE20C946F2EEC016A0119
:105640007B012115310541F4E881F9810190F08158
:10565000E02D642F09951DC02A303105A9F477FF8C
:1056600012C06DE20E948A2A8C0144275527BA0194
:105670004C195D096E097F092AE0CE010E94DC2ADF
:10568000800F911F06C02AE0B701A601CE010E943B
:10569000DC2ACDB7DEB7E8E00C948B2E9A01AB0183
:1056A000662757FD6095762F0E94182B08950F935B
:1056B0001F93CF93DF93EC019A01AB01662757FD4F
:1056C0006095762F0E94182B8C01CE010E94922AA1
:1056D000800F911FDF91CF911F910F910895211598
:1056E000310549F4DC01ED91FC910190F081E02D50
:1056F000642F099508950E94DC2A08959A01462F87
:1057000050E060E070E00E946F2B08959A01AB01B9
:1057100060E070E00E946F2B08950F931F93CF936A
:10572000DF93EC010E946F2B8C01CE010E94922A24
:10573000800F911FDF91CF911F910F9108950F93CB
:105740001F93CF93DF93EC019A01AB0160E070E00F
:105750000E946F2B8C01CE010E94922A800F911F14
:10576000DF91CF911F910F9108950F931F93CF93C6
:10577000DF93EC019A01462F50E060E070E00E9458
:105780006F2B8C01CE010E94922A800F911FDF9116
:10579000CF911F910F910895FC0124853585F90162
:1057A000E05CFF4F80819181F901EE5BFF4F20812A
:1057B0003181821B930B8F7399270895FC01848597
:1057C0009585FC01E05CFF4F40815181FC01EE5B5F
:1057D000FF4F208131814217530741F00190F08142
:1057E000E02DE80FF91F808190E008958FEF9FEF83
:1057F0000895FC0184859585FC01E05CFF4F4081A4
:105800005181FC01EE5BFF4F20813181421753072C
:1058100079F0A081B181A80FB91F8C9120813181CD
:105820002F5F3F4F2F7333273183208390E00895FC
:105830008FEF9FEF0895FC0181A1882329F0A489AF
:10584000B5898C9186FFFBCF11A20895CF93DF938A
:10585000FC0126853785D901A05CBF4F8D919C91B5
:10586000119701968F739927E901CE5BDF4F48812D
:10587000598184179507D9F30D90BC91A02DA20FE3
:10588000B31F6C93A685B785A05CBF4F11969C9300
:105890008E93A689B7892C9181E090E0078C02C095
:1058A000880F991F0A94E2F7282B2C9381E081A39B
:1058B0000488F589E02D80818064808381E090E018
:1058C000DF91CF91089508951F920F920FB60F9216
:1058D00011242F933F934F938F939F93EF93FF93B5
:1058E0008091C00082FD1CC04091C6008091880656
:1058F0009091890601968F73992720918A0630919D
:105900008B068217930771F0E0918806F091890663
:10591000E85BF94F4083909389068093880602C024
:105920008091C600FF91EF919F918F914F913F9190
:105930002F910F900FBE0F901F90189582EE95E05B
:105940000E94CC2B892B11F00E94632C08951F928A
:105950000F920FB60F9211242F933F938F939F9323
:10596000EF93FF93209144063091450680914606BF
:10597000909147062817390731F48091C1008F7D37
:105980008093C10014C0E0914606F0914706EC5F99
:10599000F94F2081809146069091470601968F73BA
:1059A000992790934706809346062093C600FF915F
:1059B000EF919F918F913F912F910F900FBE0F907C
:1059C0001F901895A0E0B0E0E8EEFCE20C946B2E7E
:1059D000FC011382128288EE93E0A0E0B0E08483A1
:1059E0009583A683B7838CEB93E09183808375873F
:1059F000648757874687318B208B138B028BF58A00
:105A0000E48AD78AC68AB18EA08E938E828E8F85C5
:105A1000848F8889858F8989868F8A89878F8B89EA
:105A200080A3ECE00C94872ECF92DF92EF92FF924E
:105A3000CF93DF93EC016A017B01411581EE58079A
:105A400061057105F9F0EC89FD8981E090E008A01D
:105A500002C0880F991F0A94E2F7808360E079E022
:105A60008DE390E0A70196010E94242E2150310978
:105A7000410951095695479537952795211580E19C
:105A8000380798F0EC89FD89108260E874E88EE1AF
:105A900090E0A70196010E94242E2150310941096E
:105AA00051095695479537952795E889F9893083A7
:105AB000EA89FB89208319A2EE89FF89408181E070
:105AC00090E09C010C8C02C0220F331F0A94E2F775
:105AD000422B4083EE89FF8940819C010D8C02C0DE
:105AE000220F331F0A94E2F7422B4083EE89FF898D
:105AF00040819C010E8C02C0220F331F0A94E2F7F2
:105B0000422B4083EE89FF8920810F8C02C0880FD1
:105B1000991F0A94E2F7809582238083DF91CF91C9
:105B2000FF90EF90DF90CF9008958F929F92AF9269
:105B3000BF92CF92DF92EF92FF920F931F9381E07B
:105B40008F9385E08F9387E08F9383E08F9384E03A
:105B50008F93E6EC8E2E912CF2ECAF2EB12CA1ECB3
:105B6000CA2ED12CB0ECEB2EF12C04EC10E025EC7D
:105B700030E044E056E068E476E082EE95E00E9492
:105B8000E22C0F900F900F900F900F901F910F919C
:105B9000FF90EF90DF90CF90BF90AF909F908F904D
:105BA00008950E9415290E948D22CEE9DCE20E9410
:105BB00021252097E1F30E949E2CF9CFA29FB001EE
:105BC000B39FC001A39F700D811D1124911DB29F31
:105BD000700D811D1124911D08950E94DE2DA59F39
:105BE000900DB49F900DA49F800D911D11240895D8
:105BF000B7FF0C94ED2D0E94ED2D821B930B0895A1
:105C0000DB018F939F930E94ED2DBF91AF91A29FD7
:105C1000800D911DA39F900DB29F900D11240895AA
:105C200097FB072E16F4009407D077FD09D00E9449
:105C3000A22E07FC05D03EF4909581959F4F0895C4
:105C4000709561957F4F0895A1E21A2EAA1BBB1B88
:105C5000FD010DC0AA1FBB1FEE1FFF1FA217B30738
:105C6000E407F50720F0A21BB30BE40BF50B661F4E
:105C7000771F881F991F1A9469F760957095809512
:105C800090959B01AC01BD01CF010895052E97FBB6
:105C90001EF400940E945D2E57FD07D00E94242E12
:105CA00007FC03D04EF40C945D2E50954095309532
:105CB00021953F4F4F4F5F4F089590958095709578
:105CC00061957F4F8F4F9F4F08952F923F924F9234
:105CD0005F926F927F928F929F92AF92BF92CF927C
:105CE000DF92EF92FF920F931F93CF93DF93CDB785
:105CF000DEB7CA1BDB0B0FB6F894DEBF0FBECDBFFD
:105D000009942A88398848885F846E847D848C84CD
:105D10009B84AA84B984C884DF80EE80FD800C81D6
:105D20001B81AA81B981CE0FD11D0FB6F894DEBFB9
:105D30000FBECDBFED010895EE0FFF1F0590F4914A
:105D4000E02D0994AA1BBB1B51E107C0AA1FBB1F72
:105D5000A617B70710F0A61BB70B881F991F5A95F7
:105D6000A9F780959095BC01CD0108958F929F92DF
:105D7000AF92BF92CF92DF92EF92FF92CF93DF93D9
:105D8000EC01688179818A819B81611571058105AA
:105D9000910521F464E279ED8BE597E02DE133EF95
:105DA00041E050E00E94462E49015A019B01AC019E
:105DB000A7EAB1E40E94ED2D6B017C01ACEEB4EFDB
:105DC000A50194010E94FB2DC60ED71EE81EF91EE8
:105DD000F7FE06C081E0C81AD108E10880E8F80A99
:105DE000C882D982EA82FB82C701B6019F77DF9120
:105DF000CF91FF90EF90DF90CF90BF90AF909F90AA
:105E00008F9008950E94B62E089586E091E00E943A
:105E1000B62E0895609306017093070180930801E0
:105E20009093090108952F923F925F926F927F9213
:105E30008F929F92AF92BF92CF92DF92EF92FF929A
:105E40000F931F93CF93DF938B01EA0161157105C7
:105E500021F0DB018C9311969C93209739F09E01E1
:105E6000225031092332310508F0D8C07C01670186
:105E7000BFEFCB1ADB0A5601F7016080862D90E058
:105E80000E944530892B11F07601F1CFFDE26F12AF
:105E90000AC0570182E0A80EB11CD70111966C9080
:105EA000772473940BC0BBE26B1207C05701E2E08A
:105EB000AE0EB11CD70111966C90712CCE018F7E65
:105EC000892B89F4B0E36B1237C0F50180818F7D97
:105ED0008835D1F46180F2E0AF0EB11C872D82606D
:105EE000782EC0E1D0E0CA30D10551F1C031D105E2
:105EF00021F0C830D10599F409C0CC24CA94DC2C17
:105F0000EC2CAFE0FA2E22C0209769F7C8E0D0E071
:105F1000CC24CA94DC2CEC2CFFE1FF2E17C06FEFD1
:105F20007FEFCB019E01442737FD4095542F0E94FF
:105F3000242E69017A010AC02097A9F6CAE0D0E0B0
:105F4000E9E9CE2EDC2CEC2CE9E1FE2EF50160E037
:105F500020E030E0A9014E01AA2497FCA094BA2CBD
:105F60001F0170ED572E560CA9E0A51570F48FEBAC
:105F7000860D8A3118F499EC592E06C08FE9860DEA
:105F80008A3148F589EA582E560C852D90E08C17F9
:105F90009D070CF56F3FD9F0C216D306E406F5064F
:105FA00098F0C501B4010E94002E9B01AC01852D23
:105FB00090E0A0E0B0E0280F391F4A1F5B1F2817B0
:105FC00039074A075B0710F46FEF01C061E03196B3
:105FD000D1016C90C5CF0115110551F0662311F068
:105FE000319703C071FE04C03297D801ED93FC9342
:105FF00070FE07C050954095309521953F4F4F4F0B
:106000005F4F67FF10C082E290E090938D0680930F
:106010008C066FEF7FEF8FEF9FEF07C060E070E0BF
:1060200080E090E002C0B901CA01DF91CF911F91D9
:106030000F91FF90EF90DF90CF90BF90AF909F9027
:106040008F907F906F905F903F902F900895FC010C
:1060500088279927E89421912032E9F3293010F01C
:106060002E30C8F32B3241F02D3239F4689404C03D
:106070000E947930820F911D219120532A30C0F364
:106080001EF4909581959F4F0895911150C08032D4
:1060900019F089508550D0F7089548EC53E00E94DC
:1060A00052300895FA01A191B081009719F4109728
:1060B000E1F0CD01DC01CD010D90002011F4C00113
:1060C00013C0FB012191222319F02015D9F7F3CF3A
:1060D000FB012191201519F41E92119606C022236E
:1060E000C1F70D900020A1F7D001FA01A193B08370
:1060F00008957AE0979F902D879F802D910D112410
:106100000895F999FECF92BD81BDF89A992780B57F
:106110000895262FF999FECF1FBA92BD81BD20BDEB
:106120000FB6F894FA9AF99A0FBE01960895992736
:0861300088270895F894FFCFC1
:1061380000008E06200001000000FF00020002009F
:106148000200020002000200020002000200020037
:106158000200020002000200020002802500000581
:10616800400AA1204EA50020244EA52C2330C012A1
:1061780000001A400AA1204EA5001B1E27522C23FE
:10618800308025000005400AA1204EA50020244E9D
:10619800A52C2330004B000006400AD0009D490082
:1061A8007B289D492C233000E1000005400A450169
:1061B800D7DC03B81E0EBF00232E48E801008A4032
:1061C8000A6001555502AD1E20000023C80154582D
:1061D8002074696D656F75742100596573004E6F81
:1061E800002C00386368004E2F41002C205B005DB6
:1061F8002028002900486F70206368616E6E656C06
:10620800200020402000456E746572696E67206129
:1062180064617074697665206368616E6E656C2070
:1062280073656C656374696F6E2C207069636B6944
:106238006E673A007363616E6E6572206D6F646598
:10624800004E4F5420454E41424C45440053656E24
:1062580064696E672073657474696E677320746F00
:106268002052580A00526573657474696E6720730A
:10627800657474696E6773206F6E2052580A004106
:10628800626F727465642065646974730A00696E6C
:1062980076616C69642073656C656374696F6E0000
:1062A8000D0A496E76616C696420696E7075742098
:1062B8002D20646973636172646564210700536506
:1062C8007474696E677320736176656420746F20D7
:1062D800454550524F4D0A005265766572746564A3
:1062E8002073657474696E67732066726F6D2045DC
:1062F8004550524F4D0A004C6F61646564206661D9
:1063080063746F72792064656661756C74730A00D2
:106318004B657920616E64206368616E6E656C738D
:106328002072616E646F6D697A65640A004F7065EA
:106338006E4C52536E67205458207374617274699E
:106348006E672000206F6E20485720006D6F6475BF
:106358006C65206C6F636B65643F00342B340038C8
:1063680000382B340031320031322B340031360002
:1063780050504D0052535349005344410053434C2D
:1063880000525844005458440041494E004C42457C
:1063980045500053504B54524D00534255530053EF
:1063A800554D44004C4C494E440000070B0C10114D
:1063B8001500B7012B032F033103350338033D03C1
:1063C800B7014003440349034D03510355035903DF
:1063D8005D0363036A036F0374038D028D028D02EC
:1063E8008D02160A1322312900000000262C2B2AC0
:0863F800CC2BF92BDE2B1B2C32
:107E00000F92CDB7DEB7112484B714BE81FFF1D035
:107E100082E08093C00088E18093C10086E0809377
:107E2000C20080E18093C4008EE0CDD088249924E4
:107E3000CC24C394F5E0DF2EE1E1EE2E73E0F72EC3
:107E4000B6D0082F813479F4B2D08983C2D0898129
:107E5000823811F481E005C0813811F485E001C059
:107E600083E09ED09AC0823411F484E103C085344B
:107E700019F485E0B6D091C0853561F498D0082F0B
:107E800010E095D090E0982E8824802A912A880CC2
:107E9000991C82C0863521F484E0A3D080E0E1CF34
:107EA000843609F04CC083D082D0A82E80D0B82E62
:107EB00000E011E07CD0F80181938F01AE16D1F77C
:107EC00088D0FB2DF53489F4E0E0F1E00BC0F9999E
:107ED000FECF92BC81BC0894811C911C819180BD15
:107EE000FA9AF99AEA1598F358C08B2D863409F05E
:107EF00054C0F401F7BEE89507B600FCFDCFF401CD
:107F0000A0E0B1E02C9130E011968C91119790E0B7
:107F1000982F8827822B932B12960C01C7BEE895C9
:107F20001124329681E0A038B80761F7F401D7BE7A
:107F3000E89507B600FCFDCFE7BEE8952EC0843774
:107F4000F1F435D034D0182F32D0B82E42D0FB2DDA
:107F5000F63421F4F40105914F010CC0FB2DF534EA
:107F600049F4F999FECF92BC81BC0894811C911C04
:107F7000F89A00B5802F14D0115049F70EC08537FC
:107F800039F427D08EE10CD085E90AD08FE069CF93
:107F9000813511F488E017D01CD080E101D050CF9A
:107FA0009091C00095FFFCCF8093C600089580910A
:107FB000C00087FFFCCF8091C00084FD01C0A89560
:107FC0008091C6000895E0E6F0E098E19083808318
:107FD0000895EDDF803219F088E0F5DFFFCF84E10E
:107FE000DFCF1F93182FE3DF1150E9F7F2DF1F9166
:0E7FF0000895282E80E0E7DFEE27FF27099492
:027FFE0001057B
:0400000300007E007B
:00000001FF
